:020000040000FA
:020000003A289C
:080008003A288C0081018316E7
:100010000313C030810508008C008101831603138F
:10002000C030810501308104831203130B110B1DB5
:1000300017288C0B162808009600051008308C0035
:100040002D2016180514161C0510960C2D208C0B4F
:10005000212805142D202D2008000C308D00332878
:1000600001308D0033288D0B332808009701382884
:100070008B10090083160313051006140113831255
:10008000031305148B100B168B1798011310180807
:1000900072209500980A18087220940013185728A7
:1000A000980A5C301802031D61281314980303306A
:1000B0009802FE301802031D612813109801980A57
:1000C000980A54301C2058301C2015081C20140895
:1000D0001C202F301C2054301C20073005200730F6
:1000E00013204728820738344B343634783432347E
:1000F000E1342E342934293437342534063422347B
:10010000793422342B3424344834283487342E3440
:1001100029343434213439343D343C3468343C346B
:10012000DE343A345934353428342E3429342634E4
:10013000A63420341A341B34EE341B342B341E34D2
:1001400045342434F1342E34293438344E34413497
:10015000673447347C344834FA34453402343B3411
:10016000B0342E3429341E348F340F34B334043475
:10017000B9340034943405348C341434CE342E34F1
:1001800029344F34F93477344534A0341E34C6341E
:0E0190001B34E434EF34F9340634FF34FF340A
:02400E00F13F80
:00000001FF
